:060000008A110A122F28EC
:10000800FF00030E83120313E700E70E0A08E80057
:100018000408E9008A110A120B1D28286D088100BE
:100028002030EE073F300318013EFF3A013EED0055
:100038000B11FF30F71B2328F607031CF707F91BE2
:100048002828F807031CF9077C08EA007D08EB005C
:100058007E08EC00282A8B1383120313850186017E
:10006800FF3083168500860006308312A000A101A8
:10007800A2018730831681004E308312ED00EE0115
:100088008100A0308B00EF01FF30F201F301F60090
:10009800F700F401F501F800F9006029F1000310F8
:1000A8006F0D723E8400831370088000840A710803
:1000B80080005E2883120313EF0A6F08023A0319BF
:1000C800EF0103106F0D8313723E84000008840A49
:1000D800000403195E28801B5E2800088A00840338
:1000E8000008820004306202031C7E28031D7E285B
:1000F80000306102031881288E280130F100003099
:10010800F0000000F00B852800000030E102031C1D
:10011800E203762800306202031C9628031D962805
:100128000430610203189928A7286208F1006108C1
:10013800F0000310F10CF00C0310F10CF00C0000AF
:10014800F00BA328000008005B085C04031DAD2821
:10015800B928F101FA30F0000000F00BB0280000D7
:100168000130DB02031CDC03A82808000515610E1A
:10017800F03986040F3886050511080085115B08DB
:10018800E100E10E0F30E105BA205B08E100BA207A
:10019800E2012830E1007620080085155B08E100BF
:1001A800E10E0F30E105BA205B08E100BA20E20158
:1001B8003230E100762008008316061286120613F4
:1001C8008613851105118312DC010F30DB00A8208E
:1001D80085110330E100BA20DC010530DB00A820DE
:1001E8000330E100BA20E2016430E10076200330F8
:1001F800E100BA20DC010530DB00A8200230E10074
:10020800BA20E2012830E10076202830DB00C22045
:100218000830DB00C2200F30DB00C2200130DB00D9
:10022800C220DC010230DB00A8200630DB00C2203F
:1002380052088A005108820053080739DB00DB0D99
:10024800DB0DDB0DF830DB054030DB04C220D601C6
:1002580008305602031C31294A295508D800540889
:1002680056070318D80AD7003D2958088A005708A6
:100278008200392183120313DB008A110A12D1206C
:10028800E2015030E1007620D60A2C2952088A0073
:10029800510882004A08D3004C08D5004B08D40006
:1002A8000130D2005930D10020298030DB00C22033
:1002B80049088A004808820007309F0001308400FE
:1002C8008407723084078313A5308000840A0330C2
:1002D80080006F08013A031D72295E280130D200A0
:1002E8007730D100E0280730CA000430CC0026302F
:1002F800CB000130C9008230C8004E290C30DB0029
:10030800C220B601B701B901031103198C298D293F
:10031800242AF1010430F0006F0884008407763045
:1003280084078313840A8017840370088000840A72
:1003380071088000A330F000013052285E28831233
:100348000313210822068A110A12031DB4296F0813
:1003580084008407763084078313840A801FA229C7
:100368002208C800210848060319BB29C429BB0173
:100378000130FF3ABB09013E0319BB0ABA00DC2968
:10038800BD01233048070318BD0A83133D1883179E
:1003980084000008C900C80A200848020318D529A3
:1003A800D629C8014808A200BB014908BA00DC29BF
:1003B8000310BB1F0314031CEC293B08BD003A08BB
:1003C8008039BC00BD013C083D04031DEC29ED2922
:1003D800FB2939083F398038DB00C2203A087F39C9
:1003E800C0004008DB00D120390A0F39B900C030FD
:1003F800DB00C2203708BD003608BC000310BD0C66
:10040800BC0C0310BD0CBC0C3C080339B80004300C
:10041800C500223038070318C50AC400172A450842
:100428008A0044088200132283120313C000400884
:10043800DB008A110A12D120B60A0319B70A8829E3
:1004480035088A00340882006C08FE006B08FD003D
:100458006A08FC006908840068088A006708830045
:10046800FF0E7F0E0900FF308312AA00FF30AD0097
:10047800FF30AB00FF30AE00FF30AC00FF30AF0004
:100488000F3083168604811304308312A900831663
:1004980023088A00220882000830B300B40104301F
:1004A8003402031C582AAF2A30083305003A031DCA
:1004B8005E2AAB2A3408340734073207B5003508FA
:1004C8003C3A0319682A6B2A2330B5007A2A350882
:1004D8003B3A0319702A732A3030B5007A2A350856
:1004E8003A3A0319782A7A2A2A30B50031083305AE
:1004F800003A031D802A812AB51783122108013E7C
:10050800FA0020087A0203188A2A8B2AFA0122089C
:100518007A060319902A962A01308316B600B6097E
:10052800B60AAB2A8316B70183122108233E831625
:100538000318B70A831383163718831784003508FE
:1005480080007A088312A1008316B601AB2A031033
:10055800B30CB40A532A2F088A002E088200A4017B
:1005680003302402031CB92A3C2B2408003A03193F
:10057800BE2AC32A8312851083168510D62A24081A
:10058800013A0319C82ACD2A8312851383168513C5
:10059800D62A2408023A0319D22AD62A8312051326
:1005A80083160513000000000000000083120608EF
:1005B800B3000608B2000608B3040608B205060828
:1005C800B3040608B2058316A7012D3024070318C3
:1005D800A70A831327188317840000088312B10021
:1005E80006088316A500A7012D3024070318A70ABB
:1005F8008313271883178400250880008312310885
:10060800831625068312B000831625088312B304C7
:10061800831625088312B20533083206B100310863
:1006280030040F39003A031D1A2B1C2B0330A90084
:1006380083162408003A0319222B272B83128514CA
:10064800831685143A2B2408013A03192C2B312BD5
:1006580083128517831685173A2B2408023A031943
:10066800362B3A2B8312051783160517A40AB42ACA
:1006780083122908003A031D422BA02BFF30A9073B
:100688002908003A0319492BA02B8316A40103302B
:100698002402031C502BA02BA7012A30240703187F
:1006A800A70A83132718831784000008A600AB0144
:1006B8002D3024070318AB0A83132B1883178400E3
:1006C800260800060F398312B0003008003A031DCF
:1006D8006E2B9D2B8316A7012D3024070318A70A1C
:1006E800831327188317840000080F39A600AB016D
:1006F8002A3024070318AB0A83132B1883178400A6
:1007080026088000831230088316B000A7012A301B
:1007180024070318A70A83132718831784000008DF
:10072800B1002408313EB2000330AF009D30AE0066
:10073800502A8316A40A4B2B831623088A00220802
:100748008200033083160313A300AE30A2008A117F
:100758000A12372A03110319B22BB32BDD2B0330EE
:100768008316A300B930A200B32AF001F101831265
:100778006F0884008407763084078313840A8017FF
:10078800840370088000840A71088000CF30F0006C
:10079800033052285E28831203136F0884008407ED
:1007A800763084078313840A8A110A12801FCE2B9D
:1007B800AE2B831621088A00200882006434003496
:1007C8000A34003410342734E834033464340034F1
:1007D8000A3400340034CA349A343B340034E134E7
:1007E800F534053480349634983400344034423437
:1007F8000F340034A03486340134003410342734E4
:1008080000340034E83403340034003464340034F1
:10081800003400340A3400340034003430343134C5
:100828003234333434343534363437343834393474
:100838004134423443344434453446347C342F34D0
:100848002D340734103408340834043402340234A4
:040858000134003433
:02400E00103F61
:00000001FF
